:030000000219FDE5
:03000B000200AA46
:03002B000201656A
:03005B000202F8A6
:030073000202DEA8
:1000800002030406080C10182030406080040608A3
:100090000C10182030406080A0C000070F1F3F0DDB
:1000A0000D04050D050305030302C2AFC0D0C0E077
:1000B000206217E5256002E473E525F4F58A758B67
:1000C00000D262D0E0D0D0D2AF3285268AC262E5BB
:1000D00026F46035306803207210758B00D0E0D0B4
:1000E000D0C293C295C297D2AF32C293C295C29783
:1000F000206E0C206609740AD5E0FDE57E429075FD
:100100008B00D0E0D0D0D2AF32758A00C28DD262DF
:1001100001FF01B9306805206602D29301B9306849
:1001200005206602D29501B9306805206602D29793
:1001300001B9C29230680A2066077408D5E0FDD282
:100140009301B9C29430680A2066077408D5E0FDAF
:10015000D29501B9C29630680A2066077408D5E0C6
:10016000FDD29701B9C2AFC2AD53E6EFC0D0C0E037
:10017000D2D3D2AFC2CEE52A6007207449152A2116
:10018000C67800790020742EE580307E01F430E3DB
:100190000278FF53DACF207E0343DA20307E034318
:1001A000DA10C2D8C271E580307E01F430E3027902
:1001B000FFC3E89970CB306103752A18207403756A
:1001C0002A18885FD27020740DE52B6004152B214E
:1001D000D643DA01C2D82070024134A85F20610200
:1001E000C2702074367982B70431C3E894F04003BA
:1001F00074F0F8E8C4540F28F87984B70302411B5F
:10020000C313C3138721200802C313200A06C3C8DF
:1002100098F8411B28F8500374FFF88822E52D5404
:10022000066011E533C313C31324062522F52250BB
:10023000037522FF7882B60459852224A824C3E5D9
:100240002495644002A864C3E895664002A86688C5
:1002500025E56970024185C3E8AA699A5003E8FA66
:10026000E4F9EAC333FBE56BF45B29400D256AF83A
:10027000E56A6002156A400B41850AC3E56A9A5037
:1002800002056A78FF8826C26EC3E52694F840020C
:10029000D26EC3E52594404002D26420CF0AD0E05C
:1002A000D0D043E610D2AD32C2CF053A7801E52A6C
:1002B0006005307402152AC3E55F9401400575623C
:1002C0000041D4756300756C00E5622401F562504D
:1002D000037562FFD0E0D0D043E610D2AD32C2AF9A
:1002E000C0D053E67FC260759100855694855795BE
:1002F000759104D0D0D2AF32C2AF53E6EFC2ADC0D9
:10030000D0C0E0C0F0D2D3D2AFA8FBA9FCC2D83095
:100310007102615F53DACF207E0343DA10307E032F
:1003200043DA20D271E580307E01F420E3026136A9
:1003300088278928A18C53DACF207E0343DA203026
:100340007E0343DA10C2D8C271307402A1787800FB
:10035000E580307E01F430E302A178885FA160532C
:10036000DACF207E0343DA20307E0343DA10C271F5
:10037000206102813853DACF207E0343DA10307EC9
:100380000343DA20C2D8D271885A895BC3E89558F2
:10039000F8E99559F97B007E087A00C3E8948CE966
:1003A00094005005755E00812A882178A2E6A82174
:1003B0006055C3E894C8E994005008E4D2E4FB7A9D
:1003C0000A8105C3E89468E994015008E4D2E3FB8C
:1003D0007A0F8105C3E894D0E994025008E4D2E290
:1003E000FB7A1E8105C3E894A0E994055008E4D285
:1003F000E1FB7A3C8105C3E89498E994085008E44D
:10040000D2E0FB7A787E00C3E8955CFCE9955DFD5F
:1004100030E70AECF42401FCEDF43400FD755E00D5
:10042000C3EC9AED9E5003755E01885C895D855A28
:1004300058855B597802A160C3E89527F8E99528AB
:10044000F9307C02A144307B02A144307A02A13D04
:10045000207502815BE9FDE8FC817AE9C313F9E8C4
:1004600013F8307902A13DE9C313F9E813F83078A5
:0F04700002A13DE9C313FDE813FC20612CC3EC8E
:10047F00941CED940240028191ED701EC3EC94C860
:10048F0050180529E52970021529C3E529940A504A
:10049F0002A178755F00D270A178E5296002152955
:1004AF007888E6F97400207F087896B90302789E61
:1004BF00E624FAFEE43400FFC3EC9EFCED9FFD92B0
:1004CF0008B90310A2085007207609D27681E330CD
:1004DF007602C276A2085016B9030DECF42401FC83
:1004EF00EDF43400FD0204FD78007900A144B90356
:1004FF0015EC33FCED33FDC3EC940AFCED9400FDD9
:10050F0050047C007D00C3EC94FFED94004006780E
:10051F00FF7900A144EC8575F0A4C5F0A2F733F87C
:10052F007900400302056078FF7900020560E9C396
:10053F0013F9E813F8307C0EE9600278FFC3E81373
:10054F0038F8E43400F9C3E894FFE99400400278E6
:10055F00FF885FD270206102A178741FF4552F4B72
:10056F00F52FC274EB7002D274752A1830740375AC
:10057F002A0A306102A18C20740353DAFE2074031F
:10058F00752B06D0F0D0E0D0D0D2AD43E610327943
:10059F00010205BC79030205BC790A0205BC791E6C
:1005AF000205BC79640205BC79C80205BC7817E462
:1005BF00D5E0FDD8FAD9F6227A147B780205E37AD2
:1005CF00107B8C0205E37A0D7BB40205E37A0B7B7B
:1005DF00C80205E37902B27DE4C294D5E0FDD2955D
:1005EF00D5E0FDC295D5E0FDD294D5E0FDD293E5DF
:1005FF0076D5E0FDC2937496D5E0FDD9D9EAF8D54A
:10060F00E0FDD8FBDBCEC29422C37C007D0075F0E9
:10061F000005F0EA33FAEB33FB50F6EB13FBEA136A
:10062F00FAC3E9FFE8FEE89AF8E99BF95004EFF9FD
:10063F00EEF8B3EC33FCED33FDD5F0DFEDF9ECF86C
:10064F0022E889F08A20D2D4F8A9F07B0030F70B8A
:10065F007BFFF42401F8E9F43400F9E88520F0A4D5
:10066F00ADF0F8E98520F0A4AFF0FEED2EF974009F
:10067F003FFA7C04C3EA13FAE913F9E813F8DCF440
:10068F008BF030F70AE8F42401F8E9F43400F9E8C4
:10069F0089F0C2D4F8A9F0227882B60403020702C7
:1006AF00C3E55F940140030206CC852224E4F5459F
:1006BF00F546F547F548F549C26D0207027882E61F
:1006CF00FCD26DE522F523783879C7AA40AB41C338
:1006DF00EB13FBEA13FAEC146013C3EB13FBEA13EF
:1006EF00FAEC14146007C3EB13FBEA13FAD1188862
:1006FF0045894622C3E5459523F8E5469400F95010
:10070F000CC3E89480E994FF4016020733C3E894C2
:10071F007FE994005003020733787F790002073393
:10072F00788079FF884A894B22E54A2547F8E54BBF
:10073F003548F9854B20E4300701F43549FA30E7A5
:10074F0009C3EA94F04015020771C3EA940F5003EE
:10075F0002077178FF79FF7A0F020771780079002D
:10076F007AF0C3E5249564500AC374019524500BA5
:10077F0002078FE54B20E70E02078FE54B30E706A8
:10078F00884789488A492278A4E6FAC3E54A33F8AC
:10079F00E54B33F9D150E930E70BC3E89480E99486
:1007AF00FF4013E1C9C3E8947FE994005002E1C907
:1007BF00787F7900E1C9788079FFE820E715C3E5F4
:1007CF002398F84009C3E8940140030207F0780129
:1007DF000207F0E8F424012523F840030207F0781C
:1007EF00FF884C2278A5E6FAA848A949D150E930EC
:1007FF00E70CC3E89401E994FF4016020824C3E80C
:10080F0094FFE99400500302082478FF790002084E
:10081F0024780179FFE920E715C3E54C98F84009E2
:10082F00C3E89401400302084B780102084BE8F437
:10083F002401254CF8400302084B78FF88242278C6
:10084F00FFC26420693D206A12D264C3E541940A55
:10085F004009C3E52594405002C26479A1E76023A3
:0D086F00E541601F74FF8541F0848539F07C
:10087C00306A0375F005A4F8C5F0600278FFC3E890
:10088C0095675002A867886622C3E5409440E5410D
:10089C009401E56650031401A6046002F566220279
:1008AC0008AE2275E890227883E6FFE5E820ECF7A5
:1008BC00A8BDA9BE0573C3E57394084052757300B7
:1008CC00E9FA79A0E76044EA7007E574601B020856
:1008DC00E9C3E895746010E5745006600C140208C6
:1008EC00F50460F90208F5E574F574C394A8401B8F
:1008FC007564C0C394054013756480C39405400BA4
:10090C00756440C39405400375640075BB0122E512
:10091C00642410500274FFF5647982B704022142FA
:10092C00C3A864E524985002A824C3E89566400245
:10093C00A86688258826E573B4070375BB1E227448
:10094C003279A687F0A4C5F0A2F733F8C3E8956412
:10095C004002A86488228824882588268867227506
:10096C0040007541F022C2AF75C820A8CCA9CDAA11
:10097C003A30CF010A75C824D2AFAB3BAC3C883BB4
:10098C00893CC3E89BF8E99C206908F9306702416F
:10099C008721E4AD3D8A3DF9EA9DFA600478FF7940
:1009AC00FFAE3EAF3F8B3E8C3FC3EC9FFCC3E99C3C
:1009BC00F542A83BA93CC3E89EF8E99FF9C3E54181
:1009CC0013FBE54013FAE82AF540E93BF5415006E4
:1009DC007540FF7541FF412EAA40AB41AC40AD4183
:1009EC007E047F02C3EB940440021E1FC3EB9408E9
:1009FC0040021E1FC3ED13FDEC13FCDEF7C3EA9C93
:100A0C00FAEB9DFBEF6009C3E913F9E813F8DFF784
:100A1C00EA28FAEB39FB8A408B4150067BFF8B406E
:100A2C008B41C3EB94025002D2673069047F0341BF
:100A3C00597892E6FFC3E537948240110FC3E5372E
:100A4C0094A040010FC3EF940640027F057E05E59C
:100A5C0041C4540FF9E541C454F0F8E540C4540FB7
:100A6C0028F8C3E89EFAE99400FB4009C3EA940213
:100A7C00EB940050047A02E4FB41D3AA40AB41EB67
:100A8C00C4FEEAC4540F4EFCC3EA9CFAEB9400FB80
:100A9C00C3E813C313F8EA28FAEB3400FB8A408B43
:100AAC0041C3EB94024002C2677805EBC4FE7B00A5
:100ABC00EAC4540F4EFAC3EA98FA4005C3940250A4
:100ACC00027A027892E6FF30600241D38552568555
:100ADC005357D26043E680C3E49AF8E49BF930673D
:100AEC0002616DE8FAE9FBD3E913FDE813FC8852C7
:100AFC008953C3EF94036038EF20E00DE82CF8E93C
:100B0C003DF9ECFAEDFB020B28E828F8E939F9C3BA
:100B1C00E82402F8E93400F97AFE7BFFC3EF940372
:100B2C00400E8A548B55884E894F8C508D5161A143
:100B3C00885489558A4E8B4F8C508D51306920C307
:100B4C00E53394034019E542A2E713F8E555F42484
:100B5C000138400B20E7087554FFF42401F555616A
:100B6C00A1E8FAD3E813FC8852C3EF94036020EF9A
:100B7C0020E007E82CF8ECFA618DE8282402F87ADA
:100B8C00FEC3EF940340088A54884E8C5061A188B0
:100B9C00548A4E8C50E56BC3335002646BF56B304A
:100BAC00600261AB753402D26043E680E52D5406D9
:100BBC006026A840A941C3E913F9E813F8C2AF5362
:100BCC00E67F759100C3E498F594E499F5957591D9
:100BDC0004D26043E680D2AF22D265754400752002
:100BEC0000306B03752040020C04D265754400750F
:100BFC002040306B03752000D2AF7801206722E5CE
:100C0C002D54066002C265C3E54194054013780279
:100C1C009405400878039405400278063069027800
:100C2C000A206019E544601530690AC3E533940362
:100C3C004003D53406D2AFD26C81DE71B3D2AF0093
:100C4C0000C2AF206726E541C3FB940F40027B0F27
:100C5C00EB240530730123306A02742820620123CF
:0E0C6C00F93069027982E58BC39940B50544E1
:100C7A00E59E7005E59B020C85E59A5440B5200275
:100C8A0081C830690A08C3E8940A400108812D2006
:100C9A0065028104C26553E67F759100306710755D
:100CAA0094007595FE759104D26043E6808104AE86
:100CBA0040AF41C3E49EF594E49FF59581AFC3E547
:100CCA00339402500281043065028104D80281DC27
:100CDA00812DC26C53E67F75910085549485559594
:100CEA00759104854E56854F57D26043E680D2AF40
:100CFA00E52D54066008206A020533020D18306C8F
:100D0A000D206B0A206507158115810215AD227821
:100D1A00003064053065027801E53775F007A4F9FB
:100D2A00E5F028F5F0E9A2F013A2F113A2F213F507
:100D3A0037C394785003753778C3E5379538400838
:100D4A00D266C293C295C297306002A152855056AC
:100D5A00855157D26043E68022207D14C2AF754385
:100D6A0002C294D292D2AF759F33759E00020F448D
:100D7A00C2AF754302C294D296D2AF759F33759EA5
:100D8A0000020F44307243207D20C2AF75430390A6
:100D9A000143757E10C297C296306204D295A1AC07
:100DAA00D294D2AF759E23020F44C2AF754303900B
:100DBA000143757E10C293C292306204D295A1CCCF
:100DCA00D294D2AF759E22020F44207D17C2AF750E
:100DDA00430390011EC297306202D295D2AF759E2C
:100DEA0023020F44C2AF75430390011EC2933062BF
:100DFA0002D295D2AF759E22020F44207D11C2AF56
:100E0A00754304C292D296D2AF759E22020F44C293
:100E1A00AF754304C296D292D2AF759E23020F4495
:100E2A00307249207D23C2AF754305900132757E29
:100E3A0004C295C294306204D293C148D292D2AF0E
:100E4A00759F33759E00020F44C2AF75430590012A
:100E5A0054757E40C295C294306204D297C16BD257
:100E6A0096D2AF759F33759E00020F44207D1AC239
:100E7A00AF754305900114C295306202D293D2AF86
:100E8A00759F33759E00020F44C2AF7543059001EA
:100E9A0028C2953062E8D297D2AF759F33759E000B
:100EAA00020F44207D11C2AF754306C296D294D276
:100EBA00AF759E23020F44C2AF754306C292D29405
:100ECA00D2AF759E22020F44307242207D20C2AFFB
:100EDA00754301900154757E40C293C292306204F8
:100EEA00D297C1F0D296D2AF759E22020F44C2AFFA
:100EFA00754301900132757E04C297C2963062042E
:100F0A00D293E110D292D2AF759E23E144207D168E
:100F1A00C2AF754301900128C293306202D297D2C0
:100F2A00AF759E22E144C2AF754301900114C29786
:100F3A00306202D293D2AF759E23C266229001120A
:100F4A00757E00C293C295C297C292C294C296C2DB
:100F5A006222788076090876090876040876FF08FE
:100F6A0076030876FF08760708760308760108767E
:100F7A0001788C76010876FF0876FF0876FF0876F6
:100F8A00FF0876FF0876030876FF0876FF0876FFE3
:100F9A000876250876D00876280876500876040858
:100FAA0076FF08760208760008767A0876FF0876D1
:100FBA0001087601087600087603227887E6FFC2E0
:100FCA0072BF0302D2727888E6C394036008C27DB6
:100FDA00E630E102D27DC27E7889E630E102D27E35
:100FEA00C3EF94026008758E01D273020FFD758EED
:100FFA0000C273227880E6149000809378A4F67871
:10100A0081E6149000809378A5F67886E61490001D
:10101A008D9378A6F6789CE67538FF75390CB4027C
:10102A00067538A075390AB403067538827539050C
:10103A0078A3E61490009A93F569120F4722227852
:10104A0096E6FA7897E6FB7888E6B40305C3EB944C
:10105A000EFB307F047A007BFFC3EB9AFCC39482B9
:0F106A0050027C827575000575EC8575F0A4C386
:10107900E5F0947D40F222D27F11491205AD7A0044
:101089007B007C101205A3E55F2AFA74003BFBDCA8
:10109900F37C04C3EB13FBEA13FADCF7FEC27F11FE
:1010A9004922E5EF20E6037520000520903DFFE584
:1010B90020146006901FFF1460009304600375EF0D
:1010C9001253D9BF7581C043FF8012059E75EF0287
:1010D90043B203E5B3240420E70DF521E5B120E08F
:1010E900068521B343B101120F4775800875A40025
:1010F90075F1FF75D4F775900275A5FC75F2FC754D
:10110900D50075A0FD75A60275F30275D60075B0F8
:10111900FF75A70175F4FF75E241E4F8F6D8FD758E
:101129006B01120F5C1215EF78988676753001C243
:10113900AF1205B71205C71205AD1205CE1205ADDE
:101149001205D51205ADC2AF78FA79FA308307D9FD
:10115900FBD8F7021C00120FC5120FFE11481149E6
:1011690078988676120F4775885075891275C82444
:1011790075910475D84075A82275B80275E6907501
:101189009B80759D00759A80759C0075D10E75BC04
:101199005875BB0175BA1F75E88012059ED2AF124A
:1011A90008AB53DACF207E0343DA20307E0343DADB
:1011B9001043DA01C2D8C2711205B7D2617B037A32
:1011C9000CE55E70077A0CDB0302114F1205AD20A6
:1011D900700302114FC270E55FC3940240E1E52F2D
:1011E900541F856160F561B560D5DAD5C26153DAFE
:1011F900CF207E0343DA20307E0343DA10C2D8C2FF
:101209007178A2E67008D274E52F54E0F52FC27503
:101219007529001205B2307409C3E529940A400200
:10122900D2751205A378023074027800C3E55F987D
:1012390040F0C2AF1205C71205C71205C7D2AF12D7
:1012490005B7754D007888E6B40302612C1205A331
:10125900788CE6C39401500302132CE530C3940142
:10126900500302132C207435C3E55F94FF50030229
:10127900132CC2AF1205DCD2AF1205B2C3E55F94DD
:101289000150EFC2AF1205C71205A81205C7D2AFA8
:101299001205B2C3E55F94FF40E90217977F02D2B6
:1012A9007F11491205B2C2AFC27F1149AE5FC3E5D2
:1012B9005F947FD2AF407612059EC2AF1205DCD291
:1012C900AFDFDC1180C3EE94057897F61205B712EB
:1012D900163112171A7F0AD27F11491205B2C2AF0D
:1012E900C27F1149AE5FC3E55F947FD2AF50E6126A
:1012F900059EC2AF1205C71205A81205C7D2AFDFF6
:10130900D61180EE24057896F61205B71216311219
:1013190017491205B21149C3E55F94FF5002416EA6
:10132900021797C3E55F954D4003855F4D1205B2DE
:1013390078017988E7B403027805C3E55F9840022C
:10134900414EC2AF1205DC1205DC1205DCD2AF1228
:1013590005B7753000E4F531F5320531E531F47042
:10136900390532789AE67819146012783214600DCA
:10137900787D14600878FA146003753200C3E53289
:1013890098401715327531B478998676C2AF12052F
:10139900DCD2AF789886761205B21205A8E52A70D4
:1013A90005307402214F78012074027806C3E55F85
:1013B9009840A77888E6C3940360031205B2E52A2A
:1013C900700302114FC2AF120F47E4F522F523F55E
:1013D90024F525F526F56AD2AF7885E6C333F56895
:1013E900E4F545F546F547F548F549F573F52CF566
:1013F9002DF53775730875BB1E12059E1208AFE5EA
:10140900E820ECFBA8BDA9BEE97001F888741208B0
:10141900B375730875BB1E7887E6FE7602120FC591
:101429007887EEF6C2AF7564FF12094B8522648591
:101439002265852266D2AF752201752401752501C1
:1014490075260185636C756D017888E6B40307C25A
:101459007D307602D27DD268D269753300120EAD25
:0F146900120ED212096B12097212096B1209725C
:1014780012096B02148BC2AF120FC5D2AF7573007D
:1014880075BB01120BF61206A7120D19120D631285
:101498000972120BE5306D03120703206703120867
:1014A8004E306703120895120D19120D8E1209722B
:1014B800120BF6306D03120738120D19120E0512B1
:1014C8000972120BE5306D03120796120D19120EF0
:1014D8002A120972120BF6306D031207F3120D1956
:1014E800120EAD1209721208AF120BE5120D191285
:1014F8000ED21208B3120972306935206B32856733
:101508006485676585636C756D0179187A0CC3E528
:101518003399400FC269D26A8A35856764856766E0
:10152800021538C3E55F9401400302148B0215B518
:10153800306A1B206B18E535147004C26A817EF589
:1015480035C3E55F9401400302148B0215B5753667
:1015580000C3E56278FA985054307404E52A604D67
:101568007888E6B40317207D05207607A1853076B4
:1015780002A185206B07D26B85676481CA78F03039
:101588006B058567647820C3E541985002818B30EC
:101598006B1BC26BC27D307602D27DD26A75351262
:1015A800856764818B0536E55F6002A1B8753600F2
:1015B800C2AF120F477887E6FE7602120FC578870A
:1015C800EEF6E4F522F523F524F525F526F568C2AF
:1015D80068D2AF12059E120F47307409C3E53694DE
:1015E800054002214F615E901A0D7820121673E5AE
:1015F80020B4550CA3121673E520B4AA03021611E1
:10160800120F5C121631021630901A0378807B0A8A
:10161800121673A308DBF9901A0F788C7B18121630
:1016280073A308DBF9901A2722C2AF1216B212165A
:101638008C901A00740E121678A37404121678A3EC
:101648007414121678901A0378807B0A121677A3FE
:1016580008DBF9901A0F788C7B18121677A308DB31
:10166800F91216C51216A3901A2722E493F622E659
:10167800438F01538FFD75EF0275B7A575B7F1F06C
:10168800538FFE22438F02438F0175EF0275B7A572
:1016980075B7F1901A0DF0538FFC22901A0D7455FE
:1016A800D178901A0E74AAD178227A3079D078201D
:1016B800901A40D173E520F709A3DAF7227A307936
:1016C800D0901A40E7D17809A3DAF922AB77A87845
:1016D800BB01027980BB02027981BB03027982BB1C
:1016E80004027984BB05027986BB06027992BB079E
:1016F800027987BB080279A3BB0902799CBB0A025D
:101708007988BB0B027989E8F7227C051205B7DCDA
:10171800FB22C2AF1205C71205CE1205D51205DC91
:101728001205A81205C71205CE1205D51205DC123E
:1017380005A81205C71205CE1205D51205DCD2AFD1
:1017480022C2AF1205DC1205D51205CE1205C7124A
:1017580005A81205DC1205D51205CE1205C712051B
:10176800A81205DC1205D51205CE1205C7D2AF2284
:10177800AE77AF78C2AF1205C71205C71205C712F8
:1017880005A8DEF21205DC1205A8DFF8D2AF22F1B7
:101798001AF112F112757701757801757900F178EF
:1017A8007C05AD5F1205B7C3ED955F70F5C3E55FC6
:1017B8009401400AC3E55F94FF40320217D3D1D4A5
:1017C800D131F11AC2AF75EF12F112DCD50579C328
:1017D800E5799403500280C6F1120578E5771490F4
:1017E800009F93F808C3E57898500280AEF112F193
:1017F800120577C3E577940C5002809C120F5C1297
:0A1808001631C2AF75EF121217126D
:0319FD000210AB2A
:101A00000E0414090904FF03FF0703010155AA018D
:101A1000FFFFFFFFFF03FFFFFF25D0285004FF0259
:081A2000007AFF01010003FF41
:101A400023506C6174696E756D31353041232020EF
:101A500023424C48454C4923463331302320202033
:101A60002020202020202020202020202020202076
:101C0000C2AFC2D353D9BF7581C043B20343FF8073
:101C1000752438752503B1C975EF0275E24043F1AB
:101C20000853A4F775D400D2837DFA780379E67C53
:101C300010752200752300901DD67B0675249875BB
:101C400025013083028142208308D8FBD9F9DCF7D3
:101C500081B4308308D8FBD9F9DCF781B4B189E4C9
:101C600093A3C39A6004DDC381B4DBDBB17B600264
:101C7000812B7B08E493FAA3B15CDBF87A30B15C8A
:101C8000752200752300B17BEAFCEBFDC3ED94FEE9
:101C9000400EB17B8A278B28ED30E0048A828B834B
:101CA000B17B7AC270D8C3ED94FE601350CEBD00F4
:101CB00025EC60097520007521FF0200008100A855
:101CC00027A9280809D804D90281D3B17FEA89AAB3
:101CD000F281C50D81A0C3ED94035049EDA2E092BD
:101CE000007AC5C3E5829400E583941C50902000DF
:101CF00010438F02438F0175B7A575B7F1F030001F
:101D00001FA827A9280809438F01538FFDD804D99C
:101D100002A12089AAE275B7A575B7F1F0A3A10DBC
:101D2000538FFC817C7AC1BD030CE493A3FAB140CC
:101D3000DCF8B138817C817EAA22AB23B15CEBFA5E
:101D4000EA6222752608C3E52313F523E52213F57D
:101D50002250066323A0632201D526EAB1C9B1C986
:101D600075260AEAF4200102D283300102C283B14F
:101D7000C9C3134002C201D526EB22B17FEAFB2082
:101D80008302A17F308302A184752608AE24AF258B
:101D9000C3EF13FFEE13FEB1CDB1C9C3EA13308315
:101DA000024480FA30E703632201C3E52313F523DD
:101DB000E52213F52250066323A0632201D526D91C
:101DC000E52265236523F52222AE24AF250E0FDE22
:101DD000FEDFFCD20122424C48656C693437316326
:041DE000F3100601F5
:00000001FF
